:102C0000120100020000004005165F810000010271
:102C100000010A0600020000004001000902200035
:102C200001010080F00904000002FF000000070518
:102C300002020002000705860200020009022000CD
:102C400001010080F00904000002FF0000000705F8
:102C50000202400000070586024000000403090448
:102C60000C03410043004300450053002603550078
:102C7000530042002D0041004900200020002000A8
:102C800020002000200020000000000000000000C4
:042C90000000000040
:1022FF006080E000013F01010101010700030202BC
:10230F0002020200F5F7F7F7F7F7F7F70000000002
:10231F000000003F013F010101010107020500001C
:10232F0000000000F6F7F7F7F7F7F7F700000000E7
:10233F000000003F011301210139010700010001D5
:10234F00000B0200FFFFFBFFFDFFFFF7003600F061
:10235F000012003F010138010101010702020D00C7
:10236F0000000000F2F7F7F7F7F7F7F700002D007E
:10237F000000003F6024E087000000000000000024
:10238F00000000000000000000000000000000003E
:10239F0000000000000000000000000047E080E0A7
:1023AF008000F7AA4E006080E0AB013F0101010100
:1023BF0001070003020202020200F5F7F7F7F7F731
:1023CF00F7F7000000000000003F013F010101018D
:1023DF0001070205000000000000F6F7F7F7F7F716
:1023EF00F7F7000000000000003F01130121013941
:1023FF00010700010001000B0200FFFFFBFFFDFFC3
:10240F00FFF7003600F0002D003F010138010101F8
:10241F00010702020D0000000000F2F7F7F7F7F7CF
:10242F00F7F700002D000000003F6024E1320000AC
:10243F00000000000000000000000000000000008D
:10244F00000000000000000000000000000000007D
:0C245F00000047E12BE08000F7AA4E00CF
:103A3D0090E60174AAF090E6F574FFF022F59B75FF
:103A4D009DE4E4F59EFF2290E67BE090E67CF00F8E
:013A5D002246
:102AB800123A3D90E12BE090E6F3F090E12CE090A3
:102AC800E6C3F090E12DE090E6C1F090E12EE090B1
:102AD800E6C2F090E130E090E6C0F090E131E0909D
:102AE800E6F4F075AF0774E0F59A74AB123A4A123F
:102AF8003A54BF80FA000000E490E6C4F0000000F9
:102B080090E6C5F090E132E090E6C6F090E133E05F
:102B180090E6C7F090E134E090E6C8F090E135E047
:102B280090E6C9F090E136E090E6CAF090E137E02F
:102B380090E6CBF090E138E090E6CCF090E139E017
:042B480090E6CDF056
:012B4C002266
:102B4D00123A3D90E080E090E6F3F090E081E09065
:102B5D00E6C3F090E082E090E6C1F090E083E09073
:102B6D00E6C2F090E085E090E6C0F090E086E0905F
:102B7D00E6F4F075AF0774E0F59A7400123A4A1254
:102B8D003A54BF80FA000000E490E6C4F000000063
:102B9D0090E6C5F090E087E090E6C6F090E088E022
:102BAD0090E6C7F090E089E090E6C8F090E08AE00A
:102BBD0090E6C9F090E08BE090E6CAF090E08CE0F2
:102BCD0090E6CBF090E08DE090E6CCF090E08EE0DA
:042BDD0090E6CDF0C1
:012BE10022D1
:0A3C4100000102020303040405055C
:10387F00EC4EFEED4F2441F582743C3EF583E4930C
:10388F00FF3395E0FEEF24A1FFEE34E68F82F58340
:10389F002290E6BCE0547EFF7E00E0D394807C0053
:0138AF0022F6
:102D2700E4F532F531F530F52FC218C215C217C2D6
:102D370016121DA2750A2C750B0075122C7513122D
:102D470075082C75091C75102C75113C75142C759C
:102D5700155CD2E843D82090E668E04409F090E695
:102D67005CE0443DF0D2AFD20C1238B090E680E080
:102D770054F7F0538EF8C2183016051224A9C2165C
:102D8700301829123BF15024C2181239AE201516FB
:102D970090E682E030E704E020E1EF90E682E03061
:102DA700E604E020E0E41238DF123C0312275B80E0
:012DB700C754
:1024A90090E6B9E0700302255A1470030225AE24A0
:1024B900FE700302260824FB7003022554147003DE
:1024C90002254E1460731460762405600302263FCA
:1024D9001229FE400302264B90E6BBE024FE60224F
:1024E90014603324FD601114602224067048E50A43
:1024F90090E6B3F0E50B8037E51290E6B3F0E5130B
:10250900802DE50C90E6B3F0E50D8023E50E90E60D
:10251900B3F0E50F801990E6BAE0FF12390BAA066D
:10252900A9077B01EA494B600DEE90E6B3F0EF9005
:10253900E6B4F002264B022644123C5F02264B12F7
:102549003C5502264B12344E02264B123C4B0226B6
:102559004B123CA4400302264B90E6B8E0247F606E
:10256900151460192402703AA215E43325E0FFA27C
:1025790017E4334F8018E490E740F080161238A032
:1025890040047D0180027D0012387FE0540190E70C
:1025990040F0E4A3F090E68AF090E68B7402F00232
:1025A900264B022644123CA6400302264B90E6B86D
:1025B900E024FE60162402600302264B90E6BAE08E
:1025C900B40105C21502264B02264490E6BAE07012
:1025D9002C1238A040047D0180027D0012387FE072
:1025E90054FEF090E6BCE05480131313541FFFE02F
:1025F900540F2F90E683F0E04420F08045803C1290
:102609003CA8503E90E6B8E024FE601A24027032DD
:1026190090E6BAE0B40104D215802790E6BAE0B496
:102629000202801E80151238A040047D0180027DBF
:102639000012387F8008120056500790E6A0E04447
:0926490001F090E6A0E04480F0ED
:012652002265
:0300330002004E7A
:04004E0053D8EF3262
:02246B00C11995
:1039890090E19EEFF0F5CB8FCDAF0590E19FEFF081
:10399900F5CA8FCCE4F5C8758E19D2BDD2AFD2ADB8
:0539A900D2CAF51C224A
:0D00360090E19EE0FF90E19FE0FD0239891E
:083C6900A21A921BD21AA21B41
:013C71002230
:083C7200A21A921CC21AA21C46
:013C7A002227
:033C9E00AF1C2236
:033CA100A21A2242
:103C1500AD07AC06C3E49DFBE49CFFEBFD023989CF
:05002E00C2CAC2AD22B0
:03002B00022BE2C3
:022BE200C0E051
:102BE400301A0E301904051C8007D219123C7BC21E
:092BF40019300303123C7BC2CF2F
:032BFD00D0E032F3
:03004300022A008E
:03005300022A007E
:102A00000239D300023A7D00023A5E000239F70033
:102A10000231690002373F0002002A000200520022
:102A2000023CAA00023CAB00023A1B00022E44000A
:102A30000234A500023CAC000234FB00023CAD00B5
:102A4000022F4D0002005200023CAE00023CAF00DB
:102A500002323800023CB00002329100023CB10068
:102A6000023CB2000200520002005200020052007A
:102A7000023CB300023CB400023CB500023CB6008C
:102A8000023CB700023CB800023CB900023CBA006C
:102A90000232EA00023CBB0002334300023CBC00AD
:102AA00002339C00023CBD000233F500023CBE0034
:082AB000023CBF00023CC00023
:1038DF0090E682E030E004E020E60B90E682E030F4
:1038EF00E119E030E71590E680E04401F07F147EA7
:0C38FF00001229B890E680E054FEF02290
:1039AE0090E682E044C0F090E681F043870100008B
:0439BE0000000022E3
:1038B000300C0990E680E0440AF0800790E680E052
:1038C0004408F07FDC7E051229B890E65D74FFF0B5
:0F38D00090E65FF05391EF90E680E054F7F0221E
:02390B00A9070A
:10390D00AE14AF158F828E83A3E064037017AD01E3
:10391D0019ED7001228F828E83E07C002FFDEC3E2D
:09392D00FEAF0580DF7E007F0083
:01393600226E
:1029B8008E378F3890E600E054187012E5382401FD
:1029C800FFE43537C313F537EF13F538801590E674
:1029D80000E05418FFBF100BE53825E0F538E5375F
:1029E80033F537E5381538AE37700215374E6005C0
:0629F8001239C280EE223C
:1039C2007400F58690FDA57C05A3E582458370F918
:0139D20022D2
:1019BB00253032625800253034580020213D20005C
:1019CB000D004020504F535420002D2050415353B5
:1019DB00200D002D204641494C200D00362D31366F
:1019EB004100362D31364500322D31364100322D36
:1019FB00313600322D31364500362D313646003624
:101A0B002D36344D4100362D36344D4500322D36B2
:101A1B00344D4100322D36344D00322D36344D4588
:101A2B0000362D33324100362D33324500322D3303
:101A3B00324100322D333200322D33324500362DF8
:101A4B0036344100362D36344500322D36344100C4
:101A5B00322D363400322D36344500362D39364191
:101A6B0000362D39364500322D39364100322D39AD
:101A7B003600322D39364500362D3132384100369D
:101A8B002D3132384500322D3132384100322D3173
:101A9B00323800322D31323845002D4F54484552E3
:101AAB0000210054445F504F4C4C3A20475049465C
:101ABB0054524947202620307838300D005F0047BC
:101ACB005049464D6F64655365743A0020434F4E41
:101ADB0054494E554F55530D002054430D002D20A6
:101AEB003078424320577269746520002D2050696D
:101AFB00636B47504946203D2000436F6E74696EFF
:101B0B00756F757320005443204D6F646520002D55
:101B1B002057726974652034303146203D2030786F
:101B2B00002D2054436F756E74203D203078002DAE
:101B3B00204144435F436F6E74696E756F75733DDF
:101B4B00002D20435452526561640D002D204354E7
:101B5B00524D6F646520002D204354524C6F6164CD
:101B6B00200D002D204354524D6F64654C6F616402
:101B7B0020002D2044494F5772697465416C6C3AB3
:101B8B00002D2044494F5F52656164416C6C3A00F3
:101B9B002D2044494F5F436F6E6669677572653AD6
:101BAB00002D204144435F536574436F6E66696734
:101BBB003A002D204144435F476574436F6E66695D
:101BCB0067002D20307842463A476574496D6D6544
:101BDB006469617465200053746172742031204113
:101BEB00444320436F6E76657273696F6E200054A9
:101BFB00616B652032204144432C2066726573680B
:101C0B002064617461200054616B65203120414474
:101C1B00432C20686973746F726963616C20646113
:101C2B00746120002D2053656C6620546573743AE3
:101C3B00002D2050415353002D204641494C002D7F
:101C4B002050726F62652043616C3A002D205375F2
:101C5B0070706F7274656420002D20556E61766113
:101C6B00696C61626C65002D205772697465204345
:101C7B00616C200D002E0020756E617661696C61C0
:101C8B00626C652E002D2056525F4E4F53445041CF
:101C9B0055544F002D20444F204E4F542057414E4A
:101CAB0054002D2056525F52414D20262056525F34
:101CBB00454550524F4D0D002D2030784233204476
:101CCB004143446972656374200D002D20307842C6
:101CDB0033204441434D756C746944697265637478
:101CEB003A20002D204441434469726563742052AD
:101CFB006561643A0025332E31662C2025332E3155
:101D0B0066207C2025332E31662C2025332E316620
:101D1B00207C2025332E31662C2025332E31662056
:101D2B007C2025332E31662C2025332E3166002D59
:101D3B0020444143536574426F61726452616E6714
:101D4B0065002D2054445F53757370656E640D00F0
:101D5B002D2054445F526573756D650D002D205217
:101D6B00657365740031206F7574003220696E6F76
:101D7B00757400455036696E6F75740049424E009C
:101D8B004E3200706E360065663200656636004670
:071D9B004632004646360007
:10246D0041E19C0041E1C2FF41E19DFE41E1DB0004
:10247D0041E1C50042E19A0200C106C10102180006
:10248D0000C107C109C103C10BC10541E19EFB415B
:0B249D00E19F50C10402160000C100C6
:1020B600142440F58274E73CF583EFF022E0FF0537
:1020C60040E540AC3F2224A2F58274E13EF583E070
:1020D600FCA3E0FDA3E0FEA3E0227BFFE4F53C7554
:1020E6003D01227BFF753C01753D0122E538253E09
:1020F600F8E6FF7440253EF58274E7353DF5832208
:10210600E490E68AF090E6BEE090E68BF02290E658
:10211600BAE075F008A4FFA3E07C002FFFEC35F0D1
:10212600FEE42FF58274503EF583E022AD3C7AE75B
:1021360079407F40AB0722E090E740F0E490E68AE2
:10214600F090E68B22FF90E6BAE075F008A424032F
:10215600F582E5F03450F583EFF02290E65BF090DF
:10216600E65AE04401F090E65974FFF090E658E034
:102176004410F02290E6BCE0FF90E6BBE022253852
:10218600F538E53B3537F537C3E53A953CF53AE59D
:1021960039953BF5392290401C7401F0E4F09040EB
:1021A60011F022E54275F002A4246CF9742C35F086
:1021B600227586005391EF90E65D22C20890E1D722
:1021C600E0904011F022FE74402FF58274E73EF550
:1021D600832290E671F090E672F075B4FF75B6FF53
:1021E6002290E6BCE0753700F538E4F53DF53EF59E
:1021F6003DF53E2274E1F59A745AF59B74E7F59D18
:1022060074C0F59EE422904017E090E740F09040BD
:1022160018E090E741F0227B017AE1795A22C3E582
:102226003E953CE53D953B22E490E68AF090E6BE7D
:10223600E022F583E0F8A3E0F9A3E0FAA3E0FB22AD
:102246008F4A8E498D488C4722AF4AAE49AD48AC7D
:1022560047227BFF753C01E4F53D2290E60474803D
:10226600F0227BFF7A1979CB22E53EAE3D78022239
:10227600E538253EF582E537353DF583225391EF66
:1022860090E65F227BFFE4F53CF53D22F582E434DF
:1022960040F583223EF583E0FBED25E0FFEC33229B
:1022A600142440F58274E73CF583EF22F582E4348A
:1022B600E1F5832274412FF58274E73EF58322858A
:1022C6000D82850C83A37402F022850F82850E830E
:1022D600A37407F022E545AD46FCE402101AFEE0C1
:1022E6007C002400FFEC3E22EFF0053EE53E229006
:0922F60050037474F074B4F0227A
:05004600A21D9204223E
:1035F300200404E4FEFF2290E6A2E020E1F9122277
:103603001D123B91EF2401F54CE43EF54B1221FAD8
:10361300FFFEC3EF954CE54B6480F8EE6480985051
:103623000F90E67BE090E67CF00FBF00010E80E296
:09363300E54C90E68FF0AE4BFF70
:01363C00226B
:1036C2008B488A49894A200404E4FEFF221236F814
:1036D2008E518F5285484E85494F854A5012221D80
:1036E2001235511236F8745A2FF58274E13EF58381
:1036F200E4F01235F322AB48AA49A94A123B9122BF
:103BBA00200404E4FEFF2290E15AEFF0E4A3F0129D
:033BCA0035F322AE
:103AD700200404E4FEFF22754BFF754C19754DBB9E
:0C3AE7008F4E12221D1215A81235F3227A
:103A9C00200404E4FEFF22754BFF754C19754DC1D3
:0E3AAC008E4E8F4F12221D1215A81235F322D6
:1031000090E685E02405F56A200404E4FEFF2278B9
:103110005A7CE17D0112152F90E6A2E030E1079084
:06312000E685E0B56AF24D
:1031260012221D123B91EF2401F56EE43EF56D125D
:1031360021FAF56BF56CC3E56C956EE56D6480F868
:10314600E56B648098501290E67BE090E67CF00593
:103156006CE56C70E1056B80DDE56E90E68FF0AE98
:023166006DFFFB
:013168002244
:1037020075440390E1DC7430F0E4A3F0A374031277
:10371200372C7F0F123B0F90E1DC7438F0E4A3F0FA
:0A372200A30412372C7F0F023B0FA7
:10372C00F07AE17BDCAD447F0E123B0F7AE17BDC5F
:03373C00AD442277
:062ECD008F448D458B4689
:102ED3002006061222DB022F3B1222DBE54475F0AB
:102EE30008A424A2F582E434E1122238120E96E5F6
:102EF3004475F008A424A6F582E434E112223812C2
:102F03000DA5122246E4FBFAF9F8120F9C60094062
:102F130007E4FFFEFDFC800312224F1222467B00D2
:102F23007AFF797F7847120F9C500A7F007EFF7DDE
:102F33007F7C47800312224F12224612224F121027
:0A2F430053AD07AC06AF440231D1D4
:043C92004380022247
:043C96005380FD2238
:043C9A00638002221F
:103BCD001222610000007406F0000000E4F0000015
:023BDD000022C4
:103B7A00C20B90E61474E0F000000090E61A740993
:073B8A00F0000000023BCD3A
:103BDF001222610000007402F0000000E4F0000007
:023BEF000022B2
:1036800090E61274A0F000000090E6187411F000AB
:103690000000123BDF90E6917480F0000000F00023
:1036A0000000F0000000F000000090E6497482F095
:1036B000000000F0000000F0000000F00000000238
:0236C0003BDFEE
:063C8C00123680023B7AB3
:0F3C2500D20812219C75B3FF75B5FF1221D8226A
:0D3C340012219CD208F5B3F5B51221D8225B
:103ABA0090401C7401F0E4F01221C1E4F5B3F5B5AD
:0D3ACA0090E671F090E672F0F5B4F5B622CA
:103B2B0012219C1221C175B3FF75B5FF90E671741C
:0B3B3B00FFF090E67274801221DF2280
:07393700904010F0123C2546
:10393E00E4FEFD7801AF05EF08800103D8FDF5B177
:10394E008DB08EA08E9090401BEEF00EEE70E40DBA
:03395E00ED70E029
:013961002243
:102FBD00E4F546F547AF477801EF08800103D8FDEA
:102FCD00F5B18546A090401C7401F085904485B004
:102FDD0045E4F0E544B54606E5456547602B90E1CF
:102FED009D7401F0AF47123AD7AF46123AD77BFF27
:102FFD007A1979C61236C2AF45123AD7AF44123A92
:10300D00D71222681236C280060546E54670A6051F
:0E301D0047E54770A090E19DE0B4FE02E4F0AC
:01302B002282
:1037E5007BFF7A1979CD1236C27401123937740507
:1037F500123937123C34122FBD90E19DE07BFF70EA
:10380500067A1979D580047A1979DE1236C2904084
:0438150010E4F022A9
:062C94008B3E8A3F8940DF
:102C9A00E4F541754207123B918F431221347D01BD
:102CAA007F047E001235A390E740E04480902C0B0D
:102CBA00F090E740E0B4010C1221A98982F58374EF
:102CCA004FF005421221A98982F5837431F0054239
:102CDA00E543254225E0902C6CF0E4F541AF43EF43
:102CEA003395E0FEC3E5419FEE6480F87480985006
:102CFA002BAB3EAA3FA94085418275830012132F50
:102D0A00FDE5411221ABFAE54275F002A429F9EA80
:0C2D1A0035F08982F583EDF0054180C1A1
:012D2600228A
:1000030090401374AAF0E064AA70197455F0E06488
:10001300557011744FF0E0B44F0A7449F0E0B449DD
:07002300037F00227F012290
:10302C00120003EF14601B04705A1221347D017FCF
:10303C00037E001235A390E740E0541F90E1C2F0EC
:10304C0080421221347D027FF67E1D1235A390E75B
:10305C0040E0FF780208800123D8FDF53890E74165
:10306C00E090E1C2F01221347D017F037E00123525
:10307C00A390E740E0653860037F042290E740E0CE
:09308C00541FFF2290E1C2E0FF95
:013095002218
:103BA60090401AEDF090E1DBE53CF090E1C5E53D93
:043BB600F0022C9459
:10283F001221347D047FCC7E1D1235A37F437E434E
:10284F007D417C4490E740E0F8A3E0F9A3E0FAA3D0
:10285F00E0FBC31213F37068D2011221347D207F85
:10286F00D07E1D1235A3E4F544F545E545AE447819
:10287F0002C333CE33CED8F924401221D0E0FCA3CB
:10288F00E0FDA3E0FEA3E0FFC004C005C006C00743
:10289F00E545AE447802C333CE33CED8F924A2F542
:1028AF008274E13EF583D007D006D005D004121410
:1028BF00040545E545700205446408454470AC22A3
:1028CF00C201E4F544F545E545AE447803C333CE84
:1028DF0033CED8F9FBAA0624A2F58274E13AF58328
:1028EF001214103F80000074A62BF58274E13AF5A4
:1028FF0083121410000000000545E54570020544E1
:06290F006404454470C1A0
:01291500229F
:101DA200E4F537C202904019F090E6017480F01217
:101DB2003C8490E678E04401F0E05410FFC4540FF4
:101DC200445090E159F0E013E43390E1C4F090E61E
:101DD200007410F0904019E4F090E61074A0F090B6
:101DE200E611F000000090E612F0000000E490E638
:101DF20013F000000090E61474E0F0000000E4909C
:101E0200E615F01222610000007402F00000007476
:101E120006F0000000E4F000000090E618F0000078
:101E2200007411F000000090E61A7409F00000003E
:101E320012302C90E1C2EFF0E0FF4440902C0AF007
:101E4200EF541FB420004003022051901E54F82882
:101E52002873021EB4021EBF021ECB021ED7021E30
:101E6200E3021F01021F0D021F19021F25021F316B
:101E7200021F3F021F4D021F5B021F69021F7702F2
:101E82001F85021F93021FA1021FAF021FBD021F67
:101E9200CB021FD9021FE6021FF302200002200D0F
:101EA20002201A022027022034022041022051027D
:101EB2001EF37A1979E7122258FD02204C7A197919
:101EC200ED12228A7D0102204C7A1979F3122258EE
:101ED2007D0202204C7A1979F912228A7D030220AE
:101EE2004C7BFF7A1979FEE4F53CF53D7D04022036
:101EF2004C7BFF7A1A790412225A7D0502204C7A11
:101F02001A790A1220E97D0802204C7A1A791112F4
:101F120020E07D0902204C7A1A79181220E97D0A04
:101F220002204C7A1A791F1220E07D0B02204C7B92
:101F3200FF7A1A79251220E27D0C02204C7BFF7A6F
:101F42001A792C1220EB7D1002204C7BFF7A1A7931
:101F5200321220E27D1102204C7BFF7A1A7938126C
:101F620020EB7D1202204C7BFF7A1A793E1220E28E
:101F72007D1302204C7BFF7A1A79431220E27D14F2
:101F820002204C7BFF7A1A79491220EB7D10022045
:101F92004C7BFF7A1A794F1220E27D1102204C7B92
:101FA200FF7A1A79551220EB7D1202204C7BFF7AC0
:101FB2001A795B1220E27D1302204C7BFF7A1A7998
:101FC200601220E27D1402204C7BFF7A1A7966129D
:101FD20020EB7D1002204C7BFF7A1A796C1220E2F2
:101FE2007D1180667BFF7A1A79721220EB7D128056
:101FF200597BFF7A1A79781220E27D13804C7BFF9D
:102002007A1A797D1220E27D14803F7BFF7A1A7959
:10201200831220EB7D1080327BFF7A1A798A12209C
:10202200E27D1180257BFF7A1A79911220EB7D12D5
:1020320080187BFF7A1A79981220E27D13800B7B3D
:10204200FF7A1A799E1220E27D14123BA680097B48
:10205200FF7A1A79A5122C94E4FF74C62FF582E454
:1020620034E1F583E4F02F122292E4F00FBF15EA77
:1020720090401DE4F01237E5C20C123B4690E6C3D5
:102082007480F090E6C214F000000090E6E2740260
:10209200F043B202D215751B01123ABA904019E40C
:1020A200F090E65EE04438F0E044C4F0740112219E
:0420B2006102283F60
:10275B00E58070047F0180027F00EF90E68030E01F
:10276B0006E04408F08004E054F7F0E51B700330FA
:10277B000035E517451670067516087517FFE51732
:10278B00151770021516E51745167004F51B800F0B
:10279B00AE16AF177C027D3F121390EF20E00512AF
:1027AB003C968003123C92300B2D90401FE030E0A2
:1027BB0026C20B7BFF7A1A79AC1236C290401FE40B
:1027CB00F090E6F574FFF0C209122261E4F000000C
:1027DB0000123BCD123C9A300B59E5BB30E7547BD2
:1027EB00FF7A1A79AE1236C200000090E6AFE09085
:1027FB00E6B01222E4FED3EF9400EE94004016D321
:10280B0090E19BE09F90E19AE09E400990E648742E
:10281B0006F0000000123A9C7BFF7A1A79C8123638
:10282B00C290E698E0FF123AD790E699E0FF123A91
:03283B00D7C20BF6
:01283E002277
:10291600E4FF9040117404F0A374F0F0A37401F086
:10292600E490E6CEF000000090E6CFF000000090C4
:10293600E6D0F000000090E6D17420F000000075AB
:10294600BB06000000904019E4F01FEF600AE5BBEB
:1029560020E70500000080F2E4FDFCEDAE047802FD
:10296600C333CE33CED8F92402F58274F812229AF4
:102976001221CCEBF0EDAE047802C333CE33CED8C1
:10298600F92403F58274F812229AFE1222BAEBF0A9
:102996000DBD00010CED64104C70C0123BCD122130
:1029A600C390E1D8E0904012F090E1D9E090401356
:0129B600F030
:0129B70022FD
:10309600E4FF9040117404F0904013E4F090401E59
:1030A6007481F0E490E6CEF000000090E6CFF000E8
:1030B600000090E6D0F000000090E6BEE0C313905A
:1030C600E6D1F075BB06000000904019E4F01FEF52
:1030D600600AE5BB20E70500000080F2E4FF90E609
:1030E600BEE0FEEFC39E500F74402FF582E434E736
:0A30F600F583E4F00F80E7023BCD04
:10005600E4F541F542751B0190E6B9E0121451052D
:100066008B10058B1105C212048C2004E52104F0C7
:100076002204FF2307D23507CC38021B390D563C24
:100086000873910A64A20A64A30A57A90A24AC0158
:1000960002B20B92B30207B60D1EB708A6BA08E263
:1000A600BB0263BC05EDBE07EEBF0209C305EDD278
:1000B6000139D400C3D500DFD600000D5490E6A068
:1000C600E020E1F91221E71220F21222EE70020579
:1000D6003D6440453D70F0801A90E6A0E020E1F9CD
:1000E6001221E71220F21222EE7002053D6440450D
:1000F6003D70F01221427440F0020D56904011748A
:1001060014F01222F590E6BCE0905002F090E6BDA5
:10011600E0905002F090E6BAE0905001F090E6BB15
:10012600E0905001F0D20290E6587410F090E65A32
:100136000208FC90E6B8E020E71A90E6A0E020E18D
:10014600F990E740E0FF90E6BCE0FEE42E12229232
:10015600EF0205BAE4F53FF540A20233FF1220C5CF
:100166007002053F1222A6F090E65C1220C37002D0
:10017600053F1220B690E65A1220C37002053F12C0
:1001860020B690E65B1220C37002053F1220B6909F
:10019600E6581220C37002053F1220B690E65912A7
:1001A60020C37002053F1220B690E65E1220C3708F
:1001B60002053F1220B690E65F1220C37002053F8B
:1001C6001220B6E4F53DF53E12226FC333CE33CE90
:1001D600D8F91220CCFF121053AD0712226FC33389
:1001E600CE33CED8F92540FFE53F3E1221CCEDF0C7
:1001F600053EE53E7002053D6408453D70CA020DA8
:1002060019800C12217AFD90E6BAE0FB122ECD126F
:10021600291602089790E6B8E020E7307A1A79CADC
:10022600120D947BFF60067A1A79D780047A1A79C0
:10023600E41236C290E6BCE0600A146003020D5672
:10024600D20C8002C20C123B60020D5690E6BCE056
:10025600FFE42F122292E090E7400205BA90E6B83A
:10026600E030E703020392E4F51A041221617A1AD8
:1002760079E9120D8AD39400400A12210690E6A06D
:10028600E020E1F990E6BEE0C39404405090E740D8
:10029600E030E2297BFF7A1A79F71236C290E743FB
:1002A600E07BFF30E0067A1B790580047A1B791122
:1002B6001236C290E743E013920C123B6090E7407F
:1002C600E030E1197BFF7A1B791A1236C290E742B9
:1002D600E0FF123AD790E742E090401FF090E6BE6A
:1002E600E0600A90E740E020E0030203877BFF7AA4
:1002F6001B792C1236C290E6BBE0FF123AD790E685
:10030600BAE0FF123AD790E6BDE0FF123AD790E680
:10031600BCE0FF123AD7E5BB30E766E5AC20E0610A
:1003260012217A4FFF90E6BDE04FFF90E6BAE04F0C
:100336007003D38001C392097BFF7A1B793A123688
:10034600C2A209E433FF123AD790E6BBE090E6CEAC
:10035600F000000090E6BAE090E6CFF000000090D2
:10036600E6BDE090E6D0F0000000A209E433FF907D
:10037600E6BCE04F90E6D1F000000075BB06000039
:10038600001222681236C2D20B020D56E4F53FF572
:100396004090E6B01220C37002053F1220B600005E
:1003A6000090E6AF1220C37002053F1220B600008F
:1003B6000090E6991220C37002053F1220B6000095
:1003C6000090E6981220C37002053F1220B6000086
:1003D60000E51A5401FF90E6F4E054FE4F1220C4E3
:1003E6007002053F1220B600000090E6141220C3EA
:1003F6007002053F1220B600000090E61A1220C3D4
:100406007002053F1220B600000090E6351220C3A8
:100416007002053F1220B600000090E6341220C399
:100426007002053F1220B60000000540E540AE3FD1
:100436007002053F1424401221D0E5ACF000000004
:1004460090E6A91220C37002053F1220B6000000F4
:1004560090E6541220C37002053F1220B600000039
:1004660090E6551220C37002053F1220B600000028
:10047600300A047F0180027F001220C57002053F0A
:100486001222A60205BA7A1B794C120D8AB4020E04
:1004960090E6BBE0C4333354C012214B802690E66D
:1004A600BEE06403701E90E6BBE0FF7401A8070877
:1004B6008002C333D8FC25E044C012214B1221141C
:1004C60090E742F012211490E740F090E6BAE0750A
:1004D600F008A4FFA3E012212190E74102089E7ACA
:1004E6001B7957120D78F0020D567BFF7A1B796245
:1004F6001236C2E490E68B802490E6B8E030E7033B
:10050600020D5690E6BFE070047F0180027F0090E6
:10051600E6BEE04F60347A1B796E120D78F0122138
:100526007AC4131354037C005403FDE42DF582ECC6
:1005360012215A90E6BD12217DC413135403FDE423
:100546002DF582EC12215A020D5612210690E6A0D4
:10055600E020E1F990E6BEE064046003020D561265
:1005660022F590E742E0905002F090E743E0905089
:1005760002F090E740E0905001F090E741E09050A3
:1005860001F0020D5690E6B8E020E7107A1B797D5F
:10059600120D5890E6A0E020E1F980387BFF7A1B27
:1005A600798C1236C2904015E090E740F0904016E4
:1005B600E090E741F0E490E68A02089E7A1B799B78
:1005C600120D5890E6A0E020E1F990E742E05403CE
:1005D600904014F090E740E0904015F090E741E03D
:1005E600904016F0020D5690E6B8E030E703020799
:1005F600197BFF7A1B79AC1236C2C205122106900E
:10060600E6A0E020E1F990E740E090E1C6F09040F6
:1006160000F090E741E090E1C7F0904001F090E7EC
:1006260042E090E1C8F0904002F090E743E090E1AC
:10063600C9F0904003F090E744E090E1CAF09040A2
:1006460004F090E745E090E1CBF0904005F090E7AC
:1006560046E090E1CCF0904006F090E747E090E16C
:10066600CDF0904007F090E748E090E1CEF0904062
:1006760008F090E749E090E1CFF0904009F090E76C
:100686004AE090E1D0F090400AF090E74BE090E12C
:10069600D1F090400BF090E74CE090E1D2F0904022
:1006A6000CF090E74DE090E1D3F090400DF090E72C
:1006B6004EE090E1D4F090400EF090E74FE090E1EC
:1006C600D5F090400FF090E750E090E1D6F09040E2
:1006D60010F090E751E090E1D7F0904011F090E7EC
:1006E60052E090E1D8F0904012F090E753E090E1AC
:1006F600D9F0904013F090E1C2E0541FD394045017
:1007060003020D5690E754E090E1DAF090401DF0B8
:10071600020D567BFF7A1B79BD1236C290E1C6E008
:1007260090E740F090E1C7E090E741F090E1C8E043
:1007360090E742F090E1C9E090E743F090E1CAE02B
:1007460090E744F090E1CBE090E745F090E1CCE013
:1007560090E746F090E1CDE090E747F090E1CEE0FB
:1007660090E748F090E1CFE090E749F090E1D0E0E3
:1007760090E74AF090E1D1E090E74BF090E1D2E0CB
:1007860090E74CF090E1D3E090E74DF090E1D4E0B3
:1007960090E74EF090E1D5E090E74FF090E1D6E09B
:1007A60090E750F090E1D7E090E751F090E1D8E083
:1007B60090E752F090E1D9E090E753F090E1DAE06B
:1007C60090E75402089E90E6F574FFF090E6BCE0D0
:1007D600601090E6AFE090E698F090E6B0E090E624
:1007E60099F0123BCD020D567BFF7A1B79CD12365E
:1007F600C290E6BEE070277BFF7A1B79E21236C212
:10080600904018E0FF123AD7904017E0FF123AD70F
:100816001222681236C2904019E4F0020D3190E6B9
:10082600BEE064047BFF702D7A1B79FA1236C29003
:100836004019E4F012220C904019E4F0904017E0C1
:1008460090E742F0904018E090E743F090E68B7412
:1008560004F0020D567A1C79121236C212220C903E
:10086600E68B7402F0904019E4F0020D567BFF7A95
:100876001C792F1236C290E19DE0FF90E740F0EF21
:100886007BFF70067A1C793C80047A1C7943120D32
:100896006B90E6BFE090E68AF090E6BEE0020D318E
:1008A6007BFF7A1C794A1236C290E1DBE0FFB40185
:1008B6000890E74074BBF0800890E1C2E090E74002
:1008C600F0EF7BFFB401067A1C795780047A1C7915
:1008D60064120D6B12214204F0020D5690E6B8E048
:1008E60030E71990E6BEE0B4011290E7407401F0DB
:1008F6001237E590E68B7401F0020D567BFF20055A
:10090600107A1C79721236C2D205C20C123B46808E
:10091600077A1C79801236C290E1DBE0640160033D
:10092600020A06123B2B90E74074BBF090E6BBE050
:10093600C313FFE5B154802FF5B1E090E6C4F09003
:10094600E6BAE090E6C5F090E6BDE090E6BC12227D
:10095600E490E1A0F0A3EFF090E1A0E0FEA3E0FFB9
:100966004E7003020A17E5BB30E7EDE5AB20E1E880
:1009760090E19AE0FCA3E0FDD3EF9DEE9C4022902F
:10098600E19AE0FAA3E0FBEA90E6D0F0000000EB83
:1009960090E6D1F000000090E156ECF0A3EDF08077
:1009A6002790E1A0E0FCA3E0FDEC90E6D0F000008B
:1009B60000ED90E6D1F000000090E1A0E0FFA3E09A
:1009C60090E156CFF0A3EFF0E4F5BB000000E5BBE5
:1009D60020E7030080F8000000000090E156E0FEEA
:1009E600A3E0FFC390E1A1E09FF090E1A0E09EF0BC
:1009F600E5B1547F04FFE5B154802FF5B102095EDD
:100A06007BFF7A1C79821236C290E1C2E090E74001
:100A1600F0123ABA90E6BFE012222F020D317BFFA8
:100A26007A1C79901236C27BFF7A1C799F1236C2E5
:100A360090E6B5E054FEF090E6BFE012210790E69E
:100A4600BBE090E6B3F090E6BAE090E6B4F0020DB3
:100A56005690E1C47401F090E159E04401F07BFF47
:100A66007A1C79AD1236C290E6BAE0753700F538D1
:100A7600A3E0FEEE423790E6BEE0753900F53AA3F4
:100A8600E0FEEE423990E6B8E064C06003020B3344
:100A9600E53A45397003020D5690E6A0E020E1F9EB
:100AA600C3E53A9440E5399400500885393B853AC8
:100AB6003C8006753B00753C4090E6B9E064A37047
:100AC6003C90E6BCE0B4011BA3E0701790E6BBE0E7
:100AD60030E71090E7407403F0A37401F0A37407A5
:100AE600F0803EE4F53DF53E122224503412227683
:100AF600E01220F81222EE70EF053D80EBE4F53DA2
:100B0600F53E12222450101220F974CDF0053EE570
:100B16003E70EF053D80EB122132AF38AE3712350D
:100B2600A3122142E53CF0122184020A9690E6B80F
:100B3600E064406003020D56E53A45397003020D44
:100B460056122142F090E6A0E020E1F990E68BE013
:100B5600753B00F53C90E6B9E0B4A31EE4F53DF51F
:100B66003E122224501E1220F9E0FF122276EFF0E8
:100B7600053EE53E70EB053D80E7122132AF38AE0B
:100B8600371237B0E53C122184020B3E90E6B8E0FE
:060B960030E703020C41F0
:100B9C0090E6BDE030E60312283F90E6BDE030E77A
:100BAC0004C2068004A201920690E6BEE0701B7B94
:100BBC00FF7A1C79C31236C212210B12217AFD90D6
:100BCC00E6BAE0FB122ECD020D567BFF7A1C79D6CD
:100BDC001236C212210690E6A0E020E1F9E4F53DC0
:100BEC00F53E90E740E0F543E5437003020D56C334
:100BFC00E53E9404E53D94004003020D56E5433078
:100C0C00E023AF3EC007E53E25E0FFE53D33FE7433
:100C1C00422FF58274E73EF583E0FD1222BAE0FB29
:100C2C00D007122ECD053EE53E7002053DE543C3CF
:050C3C0013F54380B335
:100C41007A1C79EE120D946076754BFF754C1D750B
:100C51004D0090E1A21220D5F5518E508D4F8C4E52
:100C6100A31220D5F5558E548D538C52A31220D545
:100C7100F5598E588D578C56A31220D5F55D8E5C93
:100C81008D5B8C5AA31220D5F5618E608D5F8C5ED1
:100C9100A31220D5F5658E648D638C62A31220D5D5
:100CA100F5698E688D678C66A31220D5F56D8E6C03
:100CB1008D6B8C6A7B017AE779401215A88059A265
:100CC10001E43390E740F0A206E433A3F0E4A3F09B
:100CD100A3F0F53DF53E12226FC333CE33CED8F9E2
:100CE1001220CCFFC004C005C006C00712226FC38A
:100CF10033CE33CED8F92444F58274E73EF583D060
:100D010007D006D005D004121404053EE53E70025A
:100D1100053D6408453D70BE12222E80137BFF7A8B
:100D21001D793A1236C290E6B8E030E70912222E58
:100D310090E68BF0801F90E6BEE0D394004005E082
:100D410090E68BF090E19CE0448090401EF01237D9
:060D5100028002D322C360
:100D5700227BFF1236C2E490E68AF090E6BEE0906E
:100D6700E68BF0221236C27BFF7A1979CB1236C294
:100D7700227BFF1236C2E490E68BF090E6BBE09050
:100D87005003227BFF1236C290E6BEE0227BFF12A1
:070D970036C290E6BCE02229
:103BF1007BFF7A1D794D1236C27F017E001229B8F2
:023C0100D322CC
:103C03007F017E001229B87BFF7A1D795B1236C2D1
:023C1300D322BA
:0229FE00D322E2
:10344E0090E680E030E72100000090E6247402F060
:10345E00000000E490E625F0000000D20790E19A0B
:10346E007402F0A3E4F0801F000000E490E624F064
:10347E0000000090E6257440F0000000C20790E1C5
:10348E009AE4F0A37440F090E6BAE090E1C3F01233
:07349E0022681236C2D3229E
:0A3C4B0090E1C312213D04F0D322E2
:0A3C550090E6BAE090E158F0D322A7
:0A3C5F0090E15812213D04F0D32239
:023CA400D32229
:023CA600D32227
:023CA800D32225
:1039D300C0E0C083C082C085C084C086758600D223
:1039E300161221BA7401F0D086D084D085D082D04B
:0439F30083D0E0326B
:103A5E00C0E0C083C082C085C084C0861221B77406
:0F3A6E0004F0D086D084D085D082D083D0E032CF
:103A7D00C0E0C083C082C085C084C0861221B774E7
:0F3A8D0002F0D086D084D085D082D083D0E032B2
:10316900C0E0C0F0C083C082C085C084C0867586B7
:1031790000C0D075D000C000C001C002C003C004A7
:10318900C005C006C00785100C85110D1222C58522
:10319900080E85090F1222D01221BA7410F07BFF94
:1031A9007A1D7968123100D007D006D005D004D035
:1031B90003D002D001D000D0D0D086D084D085D021
:0831C90082D083D0F0D0E03287
:1039F700C0E0C083C082C085C084C086758600D2FF
:103A0700181221BA7408F0D086D084D085D082D01D
:043A170083D0E03246
:10373F00C0E0C083C082C085C084C08675860090FB
:10374F00E680E030E71285080C85090D1222C58549
:10375F00100E85110F1222D01221BA7420F0D086CC
:0B376F00D084D085D082D083D0E0321F
:01002A0032A3
:01005200327B
:013CAA0032E7
:013CAB0032E6
:103A1B00C0E0C083C082C085C084C086758600129A
:103A2B0022837404F0D086D084D085D082D083D00A
:023A3B00E03277
:102E4400C0E0C0F0C083C082C085C084C0867586DF
:102E540000C0D075D000C000C001C002C003C004CF
:062E6400C005C006C00716
:102E6A0090E68DE0FF90E6A2E020E127E4FEEEC3C3
:102E7A009F501B74802EF582E434E7F583E0FD74DD
:102E8A00C02EF582E434E7F583EDF00E80E090E69B
:102E9A008FEFF07BFF7A1D79701231001222837452
:022EAA0008F02E
:102EAC00D007D006D005D004D003D002D001D0007A
:102EBC00D0D0D086D084D085D082D083D0F0D0E052
:012ECC0032D3
:1034A500C0E0C0F0C083C082C085C084C086758678
:1034B50000C0D075D000C000C001C002C003C00468
:1034C500C005C006C0077BFF7A1D79761231001250
:1034D50022837410F0D007D006D005D004D003D0D5
:1034E50002D001D000D0D0D086D084D085D082D073
:0634F50083D0F0D0E032AC
:013CAC0032E5
:1034FB00C0E0C0F0C083C082C085C084C086758622
:10350B0000C0D075D000C000C001C002C003C00411
:10351B00C005C006C0077BFF7A1D797E12310012F1
:10352B0022837440F0D007D006D005D004D003D04E
:10353B0002D001D000D0D0D086D084D085D082D01C
:06354B0083D0F0D0E03255
:013CAD0032E4
:102F4D00C0E0C0F0C083C082C085C084C0867586D5
:102F5D0000C0D075D000C000C001C002C003C004C5
:062F6D00C005C006C0070C
:102F73005391EF751A0190E659E0F524300205C22A
:102F8300021221C37BFF7A1D798712310090E65923
:092F930074FFF090E65B7401F09C
:102F9C00D007D006D005D004D003D002D001D00089
:102FAC00D0D0D086D084D085D082D083D0F0D0E061
:012FBC0032E2
:013CAE0032E3
:013CAF0032E2
:10323800C0E0C0F0C083C082C085C084C0867586E7
:1032480000C0D075D000C000C001C002C003C004D7
:10325800C005C006C0075391EF90E65B7410F07B81
:10326800FF7A1D798B123100D007D006D005D00423
:10327800D003D002D001D000D0D0D086D084D08561
:09328800D082D083D0F0D0E032F6
:013CB00032E1
:10329100C0E0C0F0C083C082C085C084C08675868E
:1032A10000C0D075D000C000C001C002C003C0047E
:1032B100C005C006C0075391EF90E65B7440F07BF8
:1032C100FF7A1D798E123100D007D006D005D004C7
:1032D100D003D002D001D000D0D0D086D084D08508
:0932E100D082D083D0F0D0E0329D
:013CB10032E0
:013CB20032DF
:013CB30032DE
:013CB40032DD
:013CB50032DC
:013CB60032DB
:013CB70032DA
:013CB80032D9
:013CB90032D8
:013CBA0032D7
:1032EA00C0E0C0F0C083C082C085C084C086758635
:1032FA0000C0D075D000C000C001C002C003C00425
:10330A00C005C006C0075391EF90E6517402F07BE6
:10331A00FF7A1D7992123100D007D006D005D00469
:10332A00D003D002D001D000D0D0D086D084D085AE
:09333A00D082D083D0F0D0E03243
:013CBB0032D6
:10334300C0E0C0F0C083C082C085C084C0867586DB
:1033530000C0D075D000C000C001C002C003C004CB
:10336300C005C006C0075391EF90E6557402F07B89
:10337300FF7A1D7996123100D007D006D005D0040C
:10338300D003D002D001D000D0D0D086D084D08555
:09339300D082D083D0F0D0E032EA
:013CBC0032D5
:10339C00C0E0C0F0C083C082C085C084C086758682
:1033AC0000C0D075D000C000C001C002C003C00472
:1033BC00C005C006C0075391EF90E6517401F07B35
:1033CC00FF7A1D799A123100D007D006D005D004AF
:1033DC00D003D002D001D000D0D0D086D084D085FC
:0933EC00D082D083D0F0D0E03291
:013CBD0032D4
:1033F500C0E0C0F0C083C082C085C084C086758629
:1034050000C0D075D000C000C001C002C003C00418
:10341500C005C006C0075391EF90E6557401F07BD7
:10342500FF7A1D799E123100D007D006D005D00451
:10343500D003D002D001D000D0D0D086D084D085A2
:09344500D082D083D0F0D0E03237
:013CBE0032D3
:013CBF0032D2
:013CC00032D1
:06363D00AB07AA06AC0574
:10364300E4FD90E1C4E0600B7E000DEE24DC122269
:10365300B2EAF0AE050D74DC2E1222B2EBF0AF0528
:103663000D74DC2F1222B2ECF090E159E0FF7AE105
:0D3673007BDC123B0F90E159E0FF02377A3B
:0A37B0008E448F458D468A478B48F2
:1037BA00E4F549E549C3954650200545E545AE443B
:1037CA007002054414FFE5482549F582E43547F5BA
:0A37DA0083E0FD12363D054980D959
:0137E40022C2
:0A35A3008E468F478D488A498B4AF7
:1035AD00E4FDF54B90E1C4E06012E546FF7E000DB1
:1035BD00EE24DCF582E434E1F583EFF0AE050D7415
:1035CD00DC2EF582E434E1F583E547F090E159E036
:1035DD00FF7AE17BDC123B0F90E159E0FFAB4AAA89
:0635ED0049AD48023AF36B
:103B4600A20C920A90401F300A07E4F0122B4D8017
:0A3B5600067402F0122AB8023BCDFB
:103B6000A20C920A90401F300A07E4F0122B4D80FD
:0A3B7000067402F0122AB8023BCDE1
:1031D100EFC3940250047E0E80027E0FAB06EF54C3
:1031E10001FE90E67AE04401F0C2E990E678E0441D
:1031F10080F0EB25E090E679F090E678E030E0F9B8
:10320100EE441890E679F090E678E030E0F9EC9041
:10321100E679F090E678E030E0F9ED90E679F0902B
:10322100E678E04440F090E678E030E0F990E67826
:06323100E020E6F9D2E9FD
:013237002274
:093C7B000519E519700205182273
:083C8400E4F569D2E9D2AF2298
:10377A0090E678E020E6F9C2E990E678E04480F045
:10378A00EF25E090E679F090E678E030E0F990E60F
:10379A0078E04440F090E678E020E6F990E678E0B8
:0637AA0030E1D6D2E92255
:10384D00A90790E678E020E6F9E569702390E6781F
:10385D00E04480F0E925E090E679F08D64AF03A9AE
:10386D00077565018A668967E4F568756901D32274
:02387D00C32264
:10381900A90790E678E020E6F9E569702590E67851
:10382900E04480F0E925E0440190E679F08D64AF49
:1038390003A9077565018A668967E4F568756903EF
:04384900D322C322A1
:03004B0002265337
:10265300C0E0C083C082C085C084C086758600C0C8
:10266300D075D000C000C001C002C003C006C007BF
:1026730090E678E030E20675690602273D90E67839
:10268300E020E10CE5696402600675690702273DF5
:10269300E56924FE605F14603624FE700302272E72
:1026A30024FC700302273A2408600302273DAB652C
:1026B300AA66A967AF6805688F8275830012132F16
:1026C30090E679F0E56865647070756905806B90D4
:1026D300E679E0AB65AA66A967AE688E827583006A
:1026E30012136E756902E5646401704E90E678E03A
:1026F3004420F08045E56424FEB5680790E678E061
:102703004420F0E56414B5680A90E678E04440F0AC
:1027130075690090E679E0AB65AA66A967AE688E35
:102723008275830012136E0568800F90E678E0448B
:1027330040F075690080037569005391DFD007D0BD
:1027430006D003D002D001D000D0D0D086D084D020
:0827530085D082D083D0E03272
:103AF300123819E56924FA600E146006240770F37E
:0C3B0300D322E4F569D322E4F569D32253
:103B0F0012384DE56924FA600E146006240770F32D
:0C3B1F00D322E4F569D322E4F569D32237
:100D9E000210BFE86480F8E933E83360110460F0B4
:100DAE00ED33EC337009E8FCE9FDEAFEEBFF2204BB
:100DBE0060DED3EB9FEA9EE99DE8C2E78CF0C2F7B6
:100DCE0095F0400CE8CCF8E9CDF9EACEFAEBCFFB82
:100DDE0012108A85D0F05804700320D5B3E8047041
:100DEE00075002B2D50210C992D5EC0460F7E4CCDC
:100DFE00C0E0C398F8603B94186008400DD0E0FB4B
:100E0E000210A1E4FBFAC9FC8028E830E406E4C92C
:100E1E00FBE4CAFCE830E305E4C9CACBFCE854079E
:100E2E006010F8C3E913F9EA13FAEB13FBEC13FCA9
:100E3E00D8F130F52FC3E49CFCEF9BFFEE9AFEED4C
:100E4E0099FDD0E0FBEF4E4D4C701222DB030210E9
:100E5E00C6EC2CFCEF33FFEE33FEED33FDED30E749
:100E6E00EB0210A1EF2BFFEE3AFEED39FDD0E0FBC9
:100E7E0050130BBB00030210C9ED13FDEE13FEEF72
:080E8E0013FFEC13FC0210A19C
:100E9600EC4D6011E8497017ED33EC3304600DE456
:100EA600FCFFFEFD22E933E8330470F80210BF129E
:100EB600108A58046009E4CC24815006285009029F
:100EC60010C92840030210C6C0E0EB4A7044B9803E
:100ED60006D0E0FB0210B5EF4E701CBD8008EBFF9C
:100EE600EAFEE9FD80EBE98DF0A4FEE5F0020F7F56
:100EF600E9CDF9EAFEEBFFEF89F0A4FCE5F0CE8937
:100F0600F0A42EFFE435F0CD89F0A42DFEE435F0F3
:100F16008067EF4E7005BD80D780C3EF8BF0A4AC21
:100F2600F0EE8BF0A42CFCE435F0F8EF8AF0A42C5C
:100F3600E5F038FCE433CB8DF0A42CFCE5F03BF86F
:100F4600EE8AF0A42CFCE5F038F8E433CF89F0A45F
:100F56002CFCE5F038CF3400CE89F0A42FFFE5F065
:100F66003EFEE433C98DF0A42EFEE5F039CD8AF0BD
:100F7600A42FFFE5F03EFEE43DFD33D0E0FB500735
:100F86000BBB000F0210C9EC2CFCEF33FFEE33FE57
:060F9600ED33FD0210A185
:100F9C0074F8CC6480CCC86480C8F58204604FC3FC
:100FAC00EB9FF5F0EA9E42F0E99D42F0E89C45F09B
:100FBC00603C501DE5825FFFE582D313CB5BCBF425
:100FCC002B5582FB50280ABA002409B9002008804E
:100FDC001DE5825BFBE582D313CF5FCFF4C3132FE8
:100FEC005582FF50090EBE00050DBD00010CC3EB70
:100FFC009FF5F0EA9E42F0E99D42F0E89C45F060D6
:09100C0007CC4820E701B3EC22F7
:1010150075F020800E75F010800575F0087D007E56
:10102500007F003392D530D5031213E5EC33401021
:10103500EF33FFEE33FEED33FDEC33FCD5F0ED225F
:0E104500E5F0247EA2D513CC92E7CDCEFF229B
:10105300EDD2E7CD33EC3392D524814006E4FFFE95
:10106300FDFC22FCE4CFCECDCC24E0501174FF80F4
:10107300EDC3CC13CCCD13CDCE13CECF13CF047091
:07108300F030D5DE0213E599
:10154C00E55F244BF8E6055F227848301302784BB0
:10155C00E475F001121441021316200CEB7F2ED20D
:10156C000C8018EF540F2490D43440D4FF30100B5F
:10157C00EF24BFB41A0050032461FFE5606002152C
:10158C00600563E5637002056230130D7848E475FD
:10159C00F001121441EF02135C0239627403D2138E
:1015AC008003E4C213F55F8B488A49894AE4F560ED
:1015BC00F562F563E56060077F2012158780F5758D
:1015CC0061FFC20DC20CC20EC20FC211C212C214F4
:1015DC00121555FF700D3013057F00121598AF636F
:1015EC00AE6222B4255FC2D5C210121555FF24D0AD
:1015FC00B40A00501A75F00A786030D50508B6FFA9
:10160C000106C6A426F620D5047002D20F80D92478
:10161C00CFB41A00EF5004C2E5D210021885D20DD7
:10162C0080C6D20C80C0D20E80BCD2D580BAD2116A
:10163C0080B47F20121587200E077401B56000401E
:10164C00F112154CFF1215870215C0D214D212805C
:10165C009512154CFB12154CFA12154CF94A4B709D
:10166C0006797C7A197BFF200E2EE560602A7E00BD
:10167C008E8275830012132F60060EEE656170F07A
:10168C00C2D5EBC0E0EAC0E0E9C0E0EE1218E5D04C
:10169C00E0F9D0E0FAD0E0FB121316FF60AAEBC021
:1016AC00E0EAC0E0E9C0E0121587D0E02401F9D0EF
:1016BC00E03400FAD0E0FBE5610460DCD561D98050
:1016CC0087D20E80A21218C860F7E561700104126F
:1016DC0010D4A961600DE561600914F56112196FF0
:1016EC00EF60F3EA30E702F404C3995077EAF4258B
:1016FC00610430E701E404F561800D1218C860C183
:10170C00EA056125611210D4EA785EF630E701E44F
:10171C00256104D56104201101141218E5E4C0E020
:10172C0012196F785EE6601320E70714F612156F36
:10173C00802204F6D0E014C0E07F0012156FE56142
:10174C0060071215661561800B301103121566D0F7
:10175C00E00215C0D0E00480C51218C860A0E56195
:10176C00041210D4785EEAF6E561201102600104DF
:05177C0024041218E531
:1017810074FF04C0E012196F12156FE56120110298
:101791006003121566D0E0B561E87F4512157978CE
:1017A1005EE67F2B30E7047F2DF404C0E01215873D
:1017B100D0E075F00A84C0F0121570D0E0121570F7
:1017C1000215C0791080027908C212C2148008D2B1
:1017D100D5790A8004790AC2D5E561047002F56100
:1017E100E4FAFDFEFF12154CFC7B08200D131215C7
:1017F1004CFD7B10300C0A12154CFE12154CFF7B70
:1018010020EC3382D592D55013C3E4300C069FFFF0
:10181100E49EFEE4200D039DFDE49CFCE4CBF8C2B4
:101821000DEC700CCFCECDCCE824F8F870F3801716
:10183100C3EF33FFEE33FEED33FDEC33FCEB33FB53
:10184100994002FB0FD8E9EB300D05F8D0E0C44810
:10185100B20DC0E00AEC4D4E4F78207B0070C2EA19
:10186100B5610040BCC0E01218E7D0F0D0E0200D17
:1018710004C4C0E0C4B20DC0F0121570D0F0D5F0B0
:10188100EB0215C0121451165D5317C458162E4C95
:10189100162A4217C84F17D04417D0491643431789
:1018A100D65517074617654516D147199C5016326C
:1018B1002D16362E16592B163A2316572019852A1E
:1018C10015F24800001651E561B4FF037561061277
:1018D100154CFC12154CFD12154CFE12154CFF78DF
:1018E10057021103790AA2D5200F14301109B9103A
:1018F100020404B9080104A2D520120250010420F7
:101901000E68920EB560005034C0E07F20300F1990
:101911007F30A20E72127211500F12193EC20EC206
:1019210012C211C2147F30800F301103E9C0E012DE
:101931001587301103D0E0F9D0E0B560CC30111734
:101941007F30B9100C1215877F583010077F7880CF
:1019510003B90803121587300E057F2D0215877F05
:10196100202014F87F2B2012F322920E80CF7F00CB
:10197100B4070050052457F8E6FF22286E756C6CF9
:101981002900D20D12154C300DF8C20D786030D5FA
:101991000108F60215F22D5043495812154C240343
:1019A100B405004001E490199793121578743A1226
:0A19B1001578D20F7560040217C408
:10108A00E9D2E7C933E833F892D5EDD2E7CD33ECAC
:07109A0033FC5002B2D52225
:1010A100EC30E7100FBF000C0EBE00080DBD0004B0
:1010B1000BEB6014A2D5EB13FCED92E7FD2274FF5C
:1010C100FCFDFEFF22E480F8A2D574FF13FC7D80B5
:0310D100E480EFC9
:1010D400F920E72824F950037907E4F42402FB18E3
:1010E400DBFDE624FB5014E9600DE4F618E604F693
:0F10F400B40A08E4F6D9F57401F60A22C2D5222F
:10110300ED33EC3392D5FA602AB4FF33EDC2E77BBB
:10111300FF60067A117928E4227A11793120D50407
:101123007A11792C224E614E002B494E46002D49EF
:101133004E4600E47A08F608DAFC7B00740722E8DE
:10114300C0E0ECC0E0EDC0E0EEC0E0EFC0E0EA7567
:10115300F010A4CAABF075F04DA42BFBE435F0FC02
:10116300EA2410FAEB34C5FBEC34D9FCEDC2E7FFFB
:1011730075F056A4F42411C5F0F434C58FF0A42AF5
:10118300E5F03BE43CF620E7141212D6D0E0FFD0A2
:10119300E0FED0E0FDD0E0FC1212098014F404124A
:1011A30012D6D0E0FFD0E0FED0E0FDD0E0FC120E7E
:1011B30096D0E0F8E6FAEDD2E7CD33EC332482FBA8
:1011C300E4C3CF33CFCE33CECD33CD33DBF37B0785
:1011D30075F00A846004F6081B0AE5F0F6088FF040
:1011E300740AA4FFACF08EF0740AA42CFEACF05089
:1011F300010C8DF0740AA42CFDE435F0F608DBDE57
:031203007407224B
:101206000210C9EC5D046005E8590470030210BFC2
:1012160012108A580460F6EC4860F2EC7004FDFE89
:10122600FF22C860DB2481C85009C39860025006BB
:101236000210C69850CAF582E9294B4A7005AB825E
:101246000210B575F0007C1A7880C3EF9BEE9AED1C
:1012560099400DC3EF9BFFEE9AFEED99FDE842F033
:10126600DC23ACF0D0E0FFD0E0FED0E0FDAB822086
:10127600E7101BEB60BAEC2CFCEF33FFEE33FEED10
:1012860033FD0210A1E803F830E705C0F075F00061
:10129600EF2FFFEE33FEED33FD40B830E7C280AAF4
:1012A6003F8000004120000042C80000447A000050
:1012B600461C400047C35000497424004B189680D2
:1012C6004CBEBC205A0E1BCA6753C21C749DC5AEC9
:1012D600FB60065407601C2323121304EB5438608A
:1012E600091212F01212FF120E96ECF8EDF9EEFA50
:1012F600EFCB22EB1212FF80F1543803241C90121C
:10130600A6FE93FC0EEE93FD0EEE930ECE93FF22F9
:03000000022DB816
:0C2DB800787FE4F6D8FD75816E022DFFD7
:10131600BB010689828A83E0225002E722BBFE02D5
:09132600E32289828A83E4932208
:10132F00BB010CE58229F582E5833AF583E0225073
:10133F0006E92582F8E622BBFE06E92582F8E222BD
:0D134F00E58229F582E5833AF583E49322D7
:10135C00BB010689828A83F0225002F722BBFE0170
:02136C00F3226A
:10136E00F8BB010DE58229F582E5833AF583E8F0B5
:10137E00225006E92582C8F622BBFE05E92582C861
:02138E00F22249
:10139000BC000BBE0029EF8DF084FFADF022E4CC41
:1013A000F875F008EF2FFFEE33FEEC33FCEE9DEC0A
:1013B000984005FCEE9DFE0FD5F0E9E4CEFD22ED50
:1013C000F8F5F0EE8420D21CFEADF075F008EF2F9A
:1013D000FFED33FD4007985006D5F0F222C398FD8B
:0513E0000FD5F0EA2228
:0E13E500C3E49FFFE49EFEE49DFDE49CFC2219
:1013F300EB9FF5F0EA9E42F0E99D42F0E89C45F050
:0114030022C6
:0C140400ECF0A3EDF0A3EEF0A3EFF0225B
:10141000A8828583F0D083D0821214271214271259
:101420001427121427E473E493A3C583C5F0C5837E
:10143000C8C582C8F0A3C583C5F0C583C8C582C826
:011440002289
:10144100FAE6FB0808E6F925F0F618E6CA3AF622AC
:10145100D083D082F8E4937012740193700DA3A32A
:1014610093F8740193F5828883E47374029368603E
:06147100EFA3A3A380DF3E
:10396200EFB40A07740D12396D740A309811A899D0
:10397200B8130CC2983098FDA899C298B811F630C5
:0739820099FDC299F599229D
:103551008B4B8A4C894DE4F553F554E5521552AE27
:1035610051700215514E6033AB4EAA4FA950121340
:1035710016FFAB4BAA4CA94D0554E554AC53700250
:10358100055314F5828C83EF12136EEF60CD740135
:103591002550F550E4354FF54F80C0AB4BAA4CA9EF
:0235A1004D22B9
:103B9100E4FFFE121316600C0FEF70010E09E970BD
:053BA100F20A80EF2292
:10147700E709F60870FA8046E709F20870FA803E35
:1014870088828C83E709F0A370FA8074E309F60871
:1014970070FA806CE309F20870FA806488828C83A2
:1014A700E309F0A370FA805889828A83E0A3F608DB
:1014B70070FA804C89828A83E0A3F20870FA804030
:1014C70080D280FA80C680D4805180F28027801035
:1014D70080A680EA809A80A880DA80E280CA802786
:1014E70088848C8589828A83E493A30586F0A30583
:1014F7008670F5800B89828A83E493A3F60870F9D6
:10150700ECFAA9F0EDFB2288848C8589828A83E036
:10151700A30586F0A3058670F680E589828A83E4B1
:1015270093A3F20870F980D888F0ED2402B4040080
:1015370050CEF582EB2402B4040050C42323458225
:05154700239014C7739E
:102DC400022D27E493A3F8E493A34003F68001F2D1
:102DD40008DFF48029E493A3F85407240CC8C33310
:102DE400C4540F4420C8834004F456800146F6DFDF
:102DF400E4800B01020408102040809022FFE47E4E
:102E0400019360BCA3FF543F30E509541FFEE493D3
:102E1400A360010ECF54C025E060A840B8E493A39A
:102E2400FAE493A3F8E493A3C8C582C8CAC583CAC5
:102E3400F0A3C8C582C8CAC583CADFE9DEE780BE7D
:0124A8000033
:00000001FF
